:100000000C9446000C9465000C9465000C946500FB
:100010000C9465000C9465000C9465000C946500CC
:100020000C9465000C946E000C9465000C946500B3
:100030000C9465000C9465000C9465000C946500AC
:100040000C9465000C9465000C9465000C9465009C
:100050000C9465000C9465000C9465000C9465008C
:100060000C9465000C9465000C9465000C9465007C
:100070000C9465000C9465000C9465000C9465006C
:100080000C9465000C9482050C94650011241FBE2D
:10009000CFEFD0E1DEBFCDBF11E0A0E0B1E0E6EEF2
:1000A000F0E100E00BBF02C007900D92A230B10753
:1000B000D9F712E0A2E0B1E001C01D92A932B10768
:1000C000E1F70E946E010C9471080C9400008BE023
:1000D00085BD89EF83BD80E887BF08951F920F9289
:1000E0000FB60F9211248F939F93AF93BF9380917C
:1000F000020190910301A0910401B09105010196C4
:10010000A11DB11D8093020190930301A0930401EE
:10011000B0930501BF91AF919F918F910F900FBE4A
:100120000F901F90189590911C0180911D019817B8
:1001300029F480911E018F5F80931E0190931D0111
:100140000895662329F48FB5837F8FBDC79A0895DC
:1001500070E0882311F485E001C082E085BB8FB593
:100160008C608FBD709379006093780008958091C2
:100170001C01882329F480911E018F5F80931E014A
:1001800080910601909107018330910531F46091CF
:100190001E0181E00E94A1000895049729F4609156
:1001A0001E0180E00E94A100089580E887BB87E0DF
:1001B00084BB84E690E097BD86BD82E08FBD8BE175
:1001C0008EBDC79A85E085BB0895EF92FF920F938D
:1001D0001F93CF93DF93EC018B899C89029709F0E1
:1001E00076C08A818F3021F0853A09F070C047C00F
:1001F0008B81282F30E02330310531F480910601C6
:1002000090910701029749F42430310559F4809107
:10021000060190910701019791F030930701209317
:1002200006010DC0232B59F480910601909107011E
:100230000397029720F41092070110920601809113
:1002400006019091070103970297A0F410921E01F6
:1002500010921C0192E3E92EF12C04E610E021E05B
:1002600030E040E050E060E070E087EB90E00E941A
:100270003B032DC060E080E00E94A10028C0809177
:100280001C018F5F80931C01813079F482E3E82E9A
:10029000F12C00E911E021E030E040E050E060E0C6
:1002A00070E083E990E00E943B038C819B81382FB2
:1002B00020E0290F311D3093200120931F012C33A2
:1002C000310528F480911E01815080931E01DF9139
:1002D000CF911F910F91FF90EF900895EF92FF92B1
:1002E0000F931F93F8940E944D050E9467008FE0C2
:1002F0008093280260E070E080E090E00E945F055B
:1003000080E887BB87E084BB84E690E097BD86BD2C
:1003100082E08FBD8BE18EBDC79A85E085BB789466
:10032000AA9A80B58B7F80BD82B18C7F82B983B160
:10033000836083B922E3E22EF12C02E310E021E096
:1003400030E040E050E060E070E080EE91E00E943C
:100350003B030E943304FDCFDF93CF9300D0CDB792
:10036000DEB78FE08983809106018A8342E0BE0177
:100370006F5F7F4F81E00E949307882321F48CEA0E
:1003800091E00E942C050F900F90CF91DF9108957E
:10039000DF93CF930F92CDB7DEB78FE0898341E033
:1003A000BE016F5F7F4F80E20E949307882321F494
:1003B00088EC91E00E942C050F90CF91DF91089579
:1003C000EF92FF920F931F9321B130E023703070B2
:1003D0008091000190E028173907D1F132E3E32E34
:1003E000F12C01E010E021E030E040E050E060E07E
:1003F00070E08CEA91E00E943B0381B190E0837051
:1004000090708130910519F00297B9F403C082E031
:1004100090E002C081E090E0909307018093060194
:1004200087EB90E00E942C0583E990E00E942C0568
:1004300060E080E00E94A1000BC0809106019091D5
:1004400007010397029720F010920701109206010E
:1004500081B18370809300011F910F91FF90EF9005
:100460000895CF92DF92EF92FF920F931F93CF9355
:10047000DF93FC017B016901E9011A821B821C8266
:100480001D82198218829F838E83798768875B8794
:100490004A8731968FEF9FE7BF010E940D087D8745
:1004A0006C870894E11CF11C0027F7FC0095102FC5
:1004B0006FEF7FEF8FEF9FE3A80197010E94200865
:1004C000F60126873787408B518BDF91CF911F91A3
:1004D0000F91FF90EF90DF90CF900895AF92BF9271
:1004E000CF92DF92EF92FF920F931F93CF93DF9300
:1004F0005B01EA01AC01461B570B2C853D85241797
:1005000035072CF43FEFC32E3FE7D32E15C08827C5
:100510009927821B930B481759072CF421E0C22E10
:1005200020E8D22E09C08E819F81489F6001499F9B
:10053000D00C589FD00C11247A010027F7FC0095AD
:10054000102F8A819B81AC81BD81E80EF91E0A1FA4
:100550001B1F8E859F85A889B9898E159F05A007C9
:10056000B1076CF48A839B83AC83BD839FEFE92E34
:100570009FEFF92E9FEF092F9FE3192F27C0222706
:100580003327A901281B390B4A0B5B0BE216F30634
:10059000040715075CF42A833B834C835D8381E069
:1005A000E82EF12C012D80EC182F10C0EA82FB827E
:1005B0000C831D8328853985442737FD4095542FAA
:1005C000C801B7010E94EE077B018C0188819981E7
:1005D0008A199B092A853B85A901849F9001859FE3
:1005E000300D949F300D1124B982A882B60188275E
:1005F00077FD8095982F442737FD4095542F620F43
:10060000731F841F951F6E0D7F1D801F911F20E893
:1006100030E040E050E00E942008C901DA0181305A
:1006200050E895075FEFA5075FEFB50724F481E079
:1006300090E8AFEFBFEF9C01AD01203080E83807B4
:1006400080E0480780E0580724F02FEF3FE740E0C4
:1006500050E0C901DF91CF911F910F91FF90EF9072
:10066000DF90CF90BF90AF900895FC01128213826B
:10067000148215820895CF92DF92EF92FF920F932A
:100680001F93CF93DF93EC016B01A0E0B0E09A2FB2
:10069000FD0184E0EE0FFF1F8A95E1F7EA0FFB1FD3
:1006A000EF5DFE4F8785882329F09F5F1196AC3060
:1006B000B10569F7692F70E0FB01A4E0EE0FFF1FA1
:1006C000AA95E1F7E60FF71FEF5DFE4FD183C083D8
:1006D000D382C2825583448337832683E114F10495
:1006E00011F4108A08C082E3E816F10411F481E0E5
:1006F00001C082E0808BFB0134E0EE0FFF1F3A95D2
:10070000E1F7E60FF71FEF5DFE4FA089B0E0A351C0
:10071000BE4F8C91982F9E0D96878F5F8C9311877B
:10072000008781E08787F8942091020130910301CE
:100730004091040150910501C801A0E0B0E0820F92
:10074000931FA41FB51FFB0124E0EE0FFF1F2A9586
:10075000E1F7E60FF71FEF5DFE4F82879387A487CF
:10076000B5877894DF91CF911F910F91FF90EF9013
:10077000DF90CF900895CF92DF92EF92FF920F9388
:100780001F93CF93DF93DC01EB01690120E030E0A0
:10079000622FF90174E0EE0FFF1F7A95E1F7E20F87
:1007A000F31FEF5DFE4F8785882331F06F5F2F5F6A
:1007B0003F4F2C30310561F7262F30E0F90164E01E
:1007C000EE0FFF1F6A95E1F7E20FF31FEF5DFE4F9B
:1007D000B183A083D383C28355834483D782C682E7
:1007E000E114F10411F4108A08C082E3E816F10460
:1007F00011F481E001C082E0808BB90194E0660FC2
:10080000771F9A95E1F7620F731F6F5D7E4FEB01C3
:10081000E889F0E0E351FE4F8081982F9E0D9E877E
:100820008F5F80831987088781E08F87209102017D
:10083000309103014091040150910501C801A0E0ED
:10084000B0E0820F931FA41FB51FFB01828793871F
:10085000A487B587DF91CF911F910F91FF90EF9003
:10086000DF90CF900895EF92FF920F931F93CF9355
:10087000DF93F894E0900201F090030100910401ED
:100880001091050178941092F0018091F3018F5F2F
:100890008093F3018091F301883C49F48091F20147
:1008A00086958093F1011092F2011092F3014FEFBF
:1008B0005FEF20E030E0F901A4E0EE0FFF1FAA9502
:1008C000E1F7E20FF31FEF5DFE4F8785882399F074
:1008D0008091F0018F5F8093F00182859385A485DC
:1008E000B585E816F9060A071B0728F086858517DF
:1008F00010F45685422F2F5F3F4F2C303105D9F62B
:100900004F3FB9F18091F2018F5F8093F201842F04
:10091000992787FD9095EC01E4E0CC0FDD1FEA9567
:10092000E1F7C80FD91FCF5DDE4FE881F9816C81F7
:100930007D818A819B8109958E819F81892B49F4D4
:100940001F86E889F0E0E351FE4F8081815080836B
:1009500010C02A853B854C855D8588859985A0E0FA
:10096000B0E0820F931FA41FB51F8A879B87AC87B7
:10097000BD8781E0DF91CF911F910F91FF90EF90A4
:1009800008959C01DB0160E070E0FB0144E0EE0FA4
:10099000FF1F4A95E1F7E60FF71FEF5DFE4F8081DD
:1009A00091818217930719F58785882301F1F894BF
:1009B0002091020130910301409104015091050101
:1009C000CD01A0E0B0E0820F931FA41FB51FFB0173
:1009D00024E0EE0FFF1F2A95E1F7E60FF71FEF5D0A
:1009E000FE4F82879387A487B587789408956F5FB9
:1009F0007F4F6C30710549F60895AC0120E030E07E
:100A0000F901A4E0EE0FFF1FAA95E1F7E20FF31F33
:100A1000EF5DFE4F8081918184179507B9F487853A
:100A20008823A1F02091020130910301409104013B
:100A300050910501CB01A0E0B0E0820F931FA41FED
:100A4000B51F82879387A487B58708952F5F3F4F8F
:100A50002C303105A9F60895AC0120E030E0F90111
:100A6000B4E0EE0FFF1FBA95E1F7E20FF31FEF5D61
:100A7000FE4F808191818417950749F41786E0899C
:100A8000F0E0E351FE4F80818150808308952F5F15
:100A90003F4F2C30310519F7089580E090E0FC01BC
:100AA00024E0EE0FFF1F2A95E1F7E80FF91FEF5D35
:100AB000FE4F178601968C30910589F70895809135
:100AC0002802880F81608093720080E48093700018
:100AD000E1E7F0E080818C7F80832FEF209373002B
:100AE00085EC8093740081E090E09093F70180930F
:100AF000F6011092F5012093220210920C0210923E
:100B00000B0208951F920F920FB60F920BB60F9221
:100B10001124EF92FF920F931F932F933F934F93C4
:100B20005F936F937F938F939F93AF93BF93EF9355
:100B3000FF938091F6019091F701817C09F4CBC07D
:100B40008091710090E0887F90708038910561F10C
:100B500081389105ACF48836910509F48AC089364C
:100B600091052CF48036910509F0B3C09AC0803706
:100B7000910509F496C08837910509F0AAC079C09B
:100B80008039910589F0813991052CF488389105D7
:100B900009F09FC096C08839910509F492C0803A47
:100BA000910509F096C093C08091F6019091F701EC
:100BB0008034910581F4809173008093F9018FEF67
:100BC0008093220280E890E09093F7018093F601F1
:100BD0001092F5017CC08091F6019091F701803868
:100BE000910509F074C09091F5018091F901981771
:100BF000A0F48091F501E82FF0E090917300E850A7
:100C0000FE4F92838F5F8093F50190912202809135
:100C100073008927809322025AC08091F5018031A8
:100C200011F58091730080930A02909122028091C5
:100C30000A02981719F081E090E002C082E090E08B
:100C400090930C0280930B02EE24FF2400E010E04E
:100C500020E030E040E050E068EF71E085EE90E0A9
:100C60000E94BB032EC08091F5018F5F8093F50138
:100C70002EC0809126028F5F8093260280912302EE
:100C80008A3078F422E3E22EF12C02E310E020E037
:100C900030E040E050E060E070E087E597E00E94DF
:100CA000BB03809173008093F80110920C021092A4
:100CB0000B021092F50185EC8093740080E490E0C3
:100CC0007DC081E090E09093F7018093F60185EC80
:100CD000D5C085E4D3C08091710090E0887F90708A
:100CE0008032910509F49CC08132910554F4803121
:100CF000910599F088319105D1F0089709F0B7C0B6
:100D00000CC08033910509F45EC08833910509F465
:100D100060C0889709F0ABC011C080910D0280932C
:100D2000730085E88093740088E090E047C01092DB
:100D3000F40180910E02809373003BC08091F40116
:100D40008131D9F485E98093740080E290E090933A
:100D5000F7018093F6011092230280912402909172
:100D600025020196909325028093240260E070E0B2
:100D70008FE595E00E94FD0483C09091F40180917D
:100D80000E02981750F080911F028093730080919B
:100D9000F4018F5F8093F4010CC09091F401E92F6E
:100DA000F0E0E35FFD4F8281809373009F5F90933B
:100DB000F40185E88093740080E190E09093F7015E
:100DC0008093F6015DC0809126028F5F809326029A
:100DD0002CC0809126028F5F8093260260E070E035
:100DE0008FE595E00E94FD04809123028A3080F413
:100DF00092E3E92EF12C02E310E020E030E040E045
:100E000050E060E070E087E597E00E94BB0306C019
:100E100088E290E09093F7018093F60185E82EC078
:100E2000809127028F5F8093270260E070E08FE55A
:100E300095E00E94FD04809123028A3080F482E3D1
:100E4000E82EF12C02E310E020E030E040E050E03A
:100E500060E070E087E597E00E94BB0306C088E28F
:100E600090E09093F7018093F60185E907C084E054
:100E700090E09093F7018093F60185E080937400F1
:100E8000FF91EF91BF91AF919F918F917F916F9162
:100E90005F914F913F912F911F910F91FF90EF9094
:100EA0000F900BBE0F900FBE0F901F901895EF92F2
:100EB000FF920F931F938091F6019091F701019794
:100EC00071F042E3E42EF12C05E010E020E030E088
:100ED00040E050E060E070E087E597E01DC01092D0
:100EE000F40185EA8093740082E090E09093F7012A
:100EF0008093F601809123028F5F8093230232E377
:100F0000E32EF12C00E117E220E030E040E050E079
:100F100060E070E08FE595E00E943B031F910F9128
:100F2000FF90EF900895EF92FF920F931F93582F29
:100F300080912302882309F448C0809123028A30DB
:100F400009F443C081E03CC08FEF80931F02DB01B6
:100F500020E030E00DC08C91F901E35FFD4F82830A
:100F600080911F029D91892780931F022F5F3F4F21
:100F7000241788F381E080932302852F90E0880F67
:100F8000991F80930D0240930E021092F40185EA9E
:100F90008093740082E090E09093F7018093F601D3
:100FA00052E3E52EF12C05E010E020E030E040E0D7
:100FB00050E060E070E08FE595E00E943B0380E048
:100FC0001F910F91FF90EF9008958091F6019091FD
:100FD000F701019709F4B8CF82E0F2CF629FD00108
:100FE000739FF001829FE00DF11D649FE00DF11DE4
:100FF000929FF00D839FF00D749FF00D659FF00D93
:101000009927729FB00DE11DF91F639FB00DE11D7F
:10101000F91FBD01CF011124089597FB092E072662
:101020000AD077FD04D027D006D000201AF470959E
:1010300061957F4F0895F6F7909581959F4F08959C
:1010400097FB092E05260ED057FD04D028D00AD0D4
:10105000001C38F450954095309521953F4F4F4FE7
:101060005F4F0895F6F790958095709561957F4F45
:101070008F4F9F4F0895AA1BBB1B51E107C0AA1FAA
:10108000BB1FA617B70710F0A61BB70B881F991F29
:101090005A95A9F780959095BC01CD010895A1E2DC
:1010A0001A2EAA1BBB1BFD010DC0AA1FBB1FEE1FE2
:1010B000FF1FA217B307E407F50720F0A21BB30B2D
:1010C000E40BF50B661F771F881F991F1A9469F7A9
:1010D00060957095809590959B01AC01BD01CF0105
:0610E0000895F894FFCF13
:0210E600030005
:00000001FF
